S011000048656E64694374726C2E7372656396
S11300000C9434000C9451000C9451000C94510045
S11300100C9451000C9451000C9451000C94510018
S11300200C9451000C9451000C9451000C94510008
S11300300C9451000C94E0060C9451000C94510063
S11300400C9451000C9451000C9499070C948F0754
S11300500C9485070C9482000C9451000C9451006C
S11300600C9451000C94510011241FBECFEFD8E022
S1130070DEBFCDBF12E0A0E0B1E0E0E8FCE102C0E9
S113008005900D92A036B107D9F722E0A0E6B2E0C0
S113009001C01D92A13EB207E1F70E94D1020C9467
S11300A03E0E0C94000090937102809370022CE138
S11300B031E041E050E060E170E082E692E00E94CD
S11300C01E01E4E6F0E080818E7F8083EAE7F0E0C1
S11300D08081876880830895ECE7F0E09081907FC9
S11300E090648F70982B9083EAE7F0E09081986495
S11300F090838093720281E090E0909361028093F8
S1130100600208951F920F920FB60F9211242F933D
S11301103F934F935F936F937F938F939F93AF938B
S1130120BF93EF93FF93CF93DF93CDB7DEB72597BC
S1130130DEBFCDBF10926102109260028091780000
S11301402091790090917A00906190937A0092E0E6
S11301509983909172029A8390E0922B9C838B8373
S1130160BE016F5F7F4F80917002909171020E9477
S1130170630182E692E00E94F201892B51F4BE01F0
S11301806B5F7F4F82E692E00E94AC018D810E94FA
S11301906C000F900F900F900F900F90DF91CF9104
S11301A0FF91EF91BF91AF919F918F917F916F914B
S11301B05F914F913F912F910F900FBE0F901F9021
S11301C01895CF93DF931F92CDB7DEB789838091C3
S11301D0600290916102892B21F489810E946C0054
S11301E007C0BE016F5F7F4F82E692E00E94630109
S11301F00F90DF91CF910895F894809173029091BC
S1130200740201969093740280937302089580910E
S1130210730290917402892B81F080917302909102
S11302207402019790937402809373028091730215
S113023090917402892B09F4789408958F929F9277
S1130240AF92BF92CF92DF92EF92FF920F931F93E0
S1130250CF93DF93EC017B014A015901198618867B
S11302601B861A861F821E827B836A835D834C836E
S1130270CB01880F991F0E94E5089983888300E0C9
S113028010E00E151F0581F0C801880F991FC88062
S1130290D980C80ED91EC4010E94E508F6019183D5
S11302A080830F5F1F4FEDCFBD86AC86DF91CF916A
S11302B01F910F91FF90EF90DF90CF90BF90AF9080
S11302C09F908F9008950F931F93CF93DF93EC012A
S11302D08B010E94FC002E813F818A819B8128171B
S11302E0390768F5D8019D01201B310B8C819D8154
S11302F02817390780F4E885F9854D91EE0FFF1F23
S113030088819981E80FF91F80819181FC01E20FB6
S1130310F31F4083E8CF888599850196998788875C
S11303208E819F8101969F838E83288539858A815A
S11303309B812817390731F41986188603C0C0E059
S1130340D0E002C0C1E0D0E00E940701CE01DF91FD
S1130350CF911F910F9108950F931F93CF93DF9324
S1130360EC018B010E94FC008E819F81892B69F135
S1130370D801CD01801B910B2C813D8182179307FD
S113038080F4EA85FB85EE0FFF1F28813981E20F97
S1130390F31F20813181F901E80FF91F80818D93CA
S11303A0E8CF8A859B8501969B878A878E819F816A
S11303B001979F838E832A853B858A819B81281799
S11303C0390731F41B861A8603C0C0E0D0E002C0AE
S11303D0C1E0D0E00E940701CE01DF91CF911F91CF
S11303E00F910895CF93DF93EC010E94FC000E80DF
S11303F0DF81C02D0E94070181E090E0CD2B11F038
S113040080E090E0DF91CF9108958FEF8093B80062
S11304101092B900089594EA9093BC009091BC00A6
S113042097FFFCCF9091B900987F983019F085E23E
S113043091E017C0880F682B6093BB0084E8809319
S1130440BC008091BC0087FFFCCF8091B900887FFD
S1130450883129F4FA01240F351F94E805C085E397
S113046091E00E947F0B14C0E217F30789F0819199
S11304708093BB009093BC008091BC0087FFFCCFAD
S11304808091B900887F883279F387E491E0E9CFDD
S113049084E98093BC0008950F931F93CF93DF9357
S11304A000D000D0CDB7DEB78C0190937A02809350
S11304B079028091180190911901A0911A01B091CB
S11304C01B0189839A83AB83BC8380917D029091C5
S11304D07E02892BE9F0E1E0F0E00115110511F449
S11304E0E0E0F0E0EE0FFF1F81E090E08C0F9D1F35
S11304F0E80FF91F81818F9380818F938AE591E0C2
S11305009F938F930E94690B0F900F900F900F9001
S113051061E070E0012B11F460E070E087E090E0AE
S11305200F900F900F900F90DF91CF911F910F912B
S11305300C94C1060F931F93CF93DF9300D0CDB7D4
S1130540DEB78C01809375021093760280917D0250
S113055090917E02892B61F01F930F9383E791E0C2
S11305609F938F930E94690B0F900F900F900F90A1
S113057019821A8242E050E0BE016F5F7F4FC801CA
S11305800E94A6069C01AE014F5F5F4F60E080E6CB
S11305900E940B020F900F90DF91CF911F910F914A
S11305A00895CF93DF93CDB7DEB76C970FB6F89469
S11305B0DEBF0FBECDBFF894A8950FB6F894A895EA
S11305C080916000886180936000109260000FBE8B
S11305D020E231E044E050E068E070E087EC92E033
S11305E00E941E0140E052EC61E070E087EC92E072
S11305F00E94DD0742E06FEF76EF87EC92E00E9405
S1130600550787EC92E00E9453000E9405020E9465
S1130610BA068AE091E09093DC028093DB0284E3E3
S113062092E09F938F938AE392E09F938F938BE85A
S113063091E09F938F930E94690B1D8A1E8A1F8AE3
S113064043E050E0BE016B5E7F4F80E090E00E948B
S1130650AD069C01AE014B5E5F4F60E080E60E94F8
S11306600B026091DB027091DC028DE090E00E944D
S11306702D0B6091DB027091DC028AE090E00E9415
S11306802D0B6091DB027091DC028AE390E00E9402
S11306902D0B60E070E080E00E946D0760E070E088
S11306A082E00E946D0778940F900F900F900F9046
S11306B00F900F90E2E0FE2E212C312CF8EE4F2EFD
S11306C0F3E05F2E612C712CA8EB8A2EA1E09A2E08
S11306D0B2EBCB2EB1E0DB2E87EC92E00E94F2016C
S11306E0892BD1F7BE016F5E7F4F87EC92E00E94A9
S11306F0AC018989823009F431C2833009F45CC2C7
S1130700813051F78A8920917F0230918002AE01B5
S11307104F5F5F4FFA01E20FF31F10828D3009F033
S113072008C2598F488F1092800210927F02EF2CDA
S11307308F2D90E0880F991F9C01245D3D4F3B8FC6
S11307402A8F7AE9A72E71E0B72E3F2D3D7F3C8F8B
S1130750088D198DF80180818823D9F090E00E94DA
S1130760250B9C01C8010196998F888F203531058E
S113077009F055C0F80121812F3329F40E5F1F4F72
S1130780198F088F31C030E0205331092A303105E8
S1130790F0F060E177E281E00E946D076091DB0296
S11307A07091DC028DE090E00E942D0B6091DB02E1
S11307B07091DC028AE090E00E942D0B6091DB02D4
S11307C07091DC028AE390E00E942D0B72C24AE031
S11307D050E0BE01685E7F4F0E94060AE1E0FE120F
S11307E0C5C0CB010E949A026091DB027091DC02C9
S11307F08DE090E00E942D0B6091DB027091DC0291
S11308008AE090E00E942D0B809176028F93809174
S113081075028F9322E931E03F932F936AC1233508
S11308203105B1F5F80121812F3329F40E5F1F4FF3
S1130830198F088F14C030E0205331092A30310554
S113084008F0A7CF4AE050E0BE01685E7F4F0E94E7
S1130850060AE1E0FE128AC0CB010E944C026091BC
S1130860DB027091DC028DE090E00E942D0B609120
S1130870DB027091DC028AE090E00E942D0B8091F3
S11308807A028F93809179028F932CEA31E0C4CF5E
S11308902235310509F07DC0F80121812F3309F497
S11308A080C030E0205331092A30310508F071CF7F
S11308B04AE050E0BE01685E7F4F0E94060A613044
S11308C0710549F5FC8DF11151C08FEF9FE00E9435
S11308D09A0280E090E00E944C026091DB027091E9
S11308E0DC028DE090E00E942D0B6091DB027091A0
S11308F0DC028AE090E00E942D0B1F9281E08F932E
S1130900DF92CF920E94690B0F900F900F900F907F
S1130910EE24E3941DCF672B09F01ACF21E0F212E5
S113092025C08FEF9FE00E949A0280E090E00E9431
S11309304C026091DB027091DC028DE090E00E9439
S11309402D0B6091DB027091DC028AE090E00E9442
S11309502D0B1F921F92DF92CF920E94690B0F9072
S11309600F900F900F9052E0E52EF2CE6091DB02D3
S11309707091DC028DE090E00E942D0B6091DB020F
S11309807091DC028AE090E00E942D0BBF92AF923E
S1130990CBC02434310509F048C0F80121812F333C
S11309A0C9F40E5F1F4F198F088F6091DB0270919D
S11309B0DC028DE090E00E942D0B6091DB027091CF
S11309C0DC028AE090E00E942D0B81E0E81280E0D6
S11309D01F9227C030E0205331092A30310508F036
S11309E0D8CE4AE050E0BE01685E7F4F0E94060AFE
S11309F070937E0260937D026091DB027091DC0251
S1130A008DE090E00E942D0B6091DB027091DC027E
S1130A108AE090E00E942D0B80917E028F9380915A
S1130A207D028F93DF92CF9264C029343105E1F4C3
S1130A30F80181818F3309F08BCE0E5F1F4F198F20
S1130A40088F6091DB027091DC028DE090E00E94DF
S1130A502D0B6091DB027091DC028AE090E00E9431
S1130A602D0B2AE332E01EC026353105F1F4F801DE
S1130A7081818F3309F06CCE0E5F1F4F198F088F61
S1130A806091DB027091DC028DE090E00E942D0BFE
S1130A906091DB027091DC028AE090E00E942D0BF1
S1130AA024E332E03F932F9322C02435310541F5EE
S1130AB0F80181818F3309F04BCE0E5F1F4F198FE0
S1130AC0088FEA8DFB8D108101816091DB027091AA
S1130AD0DC028DE090E00E942D0B6091DB027091AE
S1130AE0DC028AE090E00E942D0B0F931F939F92EB
S1130AF08F920E94690B0F900F900F900F9028CE49
S1130B006091DB027091DC028DE090E00E942D0B7D
S1130B106091DB027091DC028AE090E00E942D0B70
S1130B202EEB31E03F932F930E94690B0F900F90AF
S1130B300FCE8A3009F4D0CD2F30310538F42F5F31
S1130B403F4F3093800220937F0280836091DB02C9
S1130B507091DC0290E00E942D0BBECD8A890B8936
S1130B601C89811116C08091770290917802081730
S1130B70190709F4B1CDF11007C0C801880F991FF6
S1130B80880F991F0E949A021093780200937702AB
S1130B90A3CD823009F0A0CD10937C0200937B0298
S1130BA081E090E00130124014F480E090E09093F2
S1130BB009018093080190CD8A89813049F118F0A8
S1130BC08230A9F189CD21E0F21203C024EF31E093
S1130BD002C028EE33E0810181E00827232819F4BC
S1130BE062E370E00BC022533109A8EEB3E00E9427
S1130BF0CB08A30192010E94A908B90180E00E94D8
S1130C006D07B80180E090E00E94C106180164CD30
S1130C1091E0F91261CD80917D0290917E02892B41
S1130C2009F491C082ED91E00E947F0B8CC062E3D5
S1130C3070E082E00E946D078091080190910901A3
S1130C4020910601309107018217930709F1209141
S1130C507D0230917E02232B61F09F938F9382EE6D
S1130C6091E09F938F930E94690B0F900F900F90C8
S1130C700F908091080190910901892B49F48FEF1D
S1130C808F0D823038F481E090E00E944C0202C063
S1130C90EF2C01C0E12C80910801909109019093FF
S1130CA007018093060180E00E94E10082E00E9437
S1130CB0E100FE1409F410CD80917D0290917E0232
S1130CC0892B01F1EE2DF0E0EE0FFF1FE45DFD4FE7
S1130CD081818F9380818F93EF2DF0E0EE0FFF1FC2
S1130CE0E45DFD4F81818F9380818F9385EF91E047
S1130CF09F938F930E94690B0F900F900F900F900A
S1130D000F900F90E2E0EE1211C08FEF9FE00E946F
S1130D109A0280E090E00E944C0261E070E082E080
S1130D2090E00E94C10692E0F92ED6CCE11008C0F2
S1130D3060E070E082E090E00E94C106F12CCCCC2F
S1130D40FF24F394C9CC82E0E82EB6CF9F70FB0158
S1130D509083818382E090E00895FB0120E4208366
S1130D6024E0880F991F2A95E1F79183828383E019
S1130D7090E008959CEF9AB986E084B99BB985B94F
S1130D800895FC01EE0FFF1F8E0F9F1FFC01E85B0F
S1130D90FD4F808121E030E0018002C0220F331F2B
S1130DA00A94E2F7428150E0E82FF0E080A1461770
S1130DB0570711F0282B02C02095282320A308955B
S1130DC01F920F920FB60F921124DF92EF92FF92AF
S1130DD00F931F932F933F934F935F936F937F933F
S1130DE08F939F93AF93BF93EF93FF93CF93DF932F
S1130DF000D000D0CDB7DEB78091C3029091C40279
S1130E009093850080938400E12CF12C93E0D92EFB
S1130E108701000F111F000F111F0D571D4FF801FF
S1130E2080819181892BF1F082819381892B31F02A
S1130E308281938101979383828314C019821A82D9
S1130E401B821C82D982EA82BE016F5F7F4F809130
S1130E508102909182020E946301892B19F0F801AA
S1130E6011821082FFEFEF1AFF0A80E1E816F10405
S1130E7079F60F900F900F900F90DF91CF91FF9123
S1130E80EF91BF91AF919F918F917F916F915F91FE
S1130E904F913F912F911F910F91FF90EF90DF9011
S1130EA00F900FBE0F901F9018959093820280931D
S1130EB081027093C4026093C302709385006093AF
S1130EC0840010928000E1E8F0E080818770482B74
S1130ED0408381E080936F0008950F931F93CF9315
S1130EE0C82F8B010E94FC0084E0C89FF0011124EC
S1130EF0ED57FD4F1383028381E090E0918380835B
S1130F00CF911F910F910C9407011F920F920FB66E
S1130F100F9211240F900FBE0F901F9018951F92DF
S1130F200F920FB60F9211240F900FBE0F901F90C7
S1130F3018951F920F920FB60F9211242F933F937F
S1130F404F935F936F937F938F939F93AF93BF93CD
S1130F50EF93FF93CF93DF9300D000D0CDB7DEB7EC
S1130F608091C00087FF12C08091C60019821A8246
S1130F701B821C8291E099838A83BE016F5F7F4F3D
S1130F808091C5029091C6020E9463010F900F9058
S1130F900F900F90DF91CF91FF91EF91BF91AF919F
S1130FA09F918F917F916F915F914F913F912F917D
S1130FB00F900FBE0F901F9018954F925F926F92F3
S1130FC07F928F929F92AF92BF92CF92DF92EF92D5
S1130FD0FF92CF93DF9300D000D0CDB7DEB76A0184
S1130FE07B019093C6028093C5024A015B0183E0B2
S1130FF0880C991CAA1CBB1C8A95D1F760E070E888
S11310008CEF9AE0A50194010E94A908CA01B901D4
S11310106B5F7F4F8F4F9F4F2AE0422E512C612CE4
S1131020712CA30192010E94A90829833A834B835E
S11310305C8334E0CC0CDD1CEE1CFF1C3A95D1F72C
S113104060E070E88CEF9AE0A70196010E94A9087D
S1131050CA01B9016B5F7F4F8F4F9F4FA30192016C
S11310600E94A90829013A01A501940169817A81A4
S11310708B819C810E949908705477FF03C07195FD
S1131080619571094B01770FAA08BB08A701960166
S1131090C301B2010E949908705477FF03C071958F
S11310A061957109CB01770FAA0BBB0B88169906C2
S11310B0AA06BB0610F0920107C029813A818091EB
S11310C0C00082608093C000215031092093C40085
S11310D03093C50088E18093C1008091C10080688D
S11310E08093C1000F900F900F900F90DF91CF91DC
S11310F0FF90EF90DF90CF90BF90AF909F908F9034
S11311007F906F905F904F9008959091C00095FFED
S1131110FCCF8093C6000895CF93C82F0E94850802
S1131120CA3019F48DE00E94850880E090E0CF91E8
S11311300895DB018F939F930E94DA08BF91AF91CA
S1131140A29F800D911DA39F900DB29F900D11241D
S11311500895A1E21A2EAA1BBB1BFD010DC0AA1FF4
S1131160BB1FEE1FFF1FA217B307E407F50720F00C
S1131170A21BB30BE40BF50B661F771F881F991F87
S11311801A9469F760957095809590959B01AC01D0
S1131190BD01CF010895A29FB001B39FC001A39FD9
S11311A0700D811D1124911DB29F700D811D11249C
S11311B0911D08950E94CB08A59F900DB49F900D9A
S11311C0A49F800D911D112408950F931F93CF9315
S11311D0DF938230910510F482E090E0E091D70231
S11311E0F091D80220E030E0A0E0B0E0309719F1AF
S11311F0408151810281138148175907C8F084172F
S1131200950769F4109731F012960C931297139680
S11312101C9327C00093D7021093D80222C0211533
S1131220310519F04217530718F49A01BD01EF0173
S1131230DF01F801DBCF21153105F9F0281B390B4B
S11312402430310580F48A819B816115710521F078
S1131250FB019383828304C09093D8028093D702C6
S1131260FE01329644C0FE01E20FF31F8193919375
S113127022503109398328833AC02091D502309114
S1131280D602232B41F420910201309103013093C3
S1131290D6022093D502209100013091010121153D
S11312A0310541F42DB73EB7409104015091050139
S11312B0241B350BE091D502F091D602E217F30717
S11312C0A0F42E1B3F0B2817390778F0AC014E5FB2
S11312D05F4F2417350748F04E0F5F1F5093D60217
S11312E04093D5028193919302C0E0E0F0E0CF01F6
S11312F0DF91CF911F910F910895CF93DF930097C2
S113130009F481C0FC01329713821282A091D702A2
S1131310B091D802109781F420813181820F931FFC
S11313202091D5023091D6022817390751F5F09350
S1131330D602E093D50267C0ED0120E030E0CE177D
S1131340DF0740F44A815B819E0141155105F1F0AC
S1131350EA01F5CFD383C28340815181840F951F65
S1131360C817D90759F488819981840F951F02966B
S1131370918380838A819B819383828321153105A4
S113138029F4F093D802E093D7023DC0E901FB832E
S1131390EA8349915991C40FD51FEC17FD0761F4F5
S11313A080819181840F951F0296E9019983888336
S11313B0828193819B838A83E0E0F0E012968D9191
S11313C09C911397009719F0FD01DC01F7CF8D91E3
S11313D09C9111979D012E5F3F4F820F931F209187
S11313E0D5023091D6022817390769F4309729F4C9
S11313F01092D8021092D70202C013821282B093C4
S1131400D602A093D502DF91CF910895A0E0B0E079
S1131410ECE0FAE00C94080E5C016B017A016115B2
S1131420710519F0FB0191838083E114F10429F023
S1131430C7010297839708F0E5C0E5012196F501FD
S11314401081812F90E00E941C0B892B11F05E010A
S1131450F4CF1D3229F42196F501118101E007C072
S11314601B3221F4E5012296F501118100E0E1141B
S1131470F10409F1F0E1EF16F10429F43FC010E39F
S1131480E114F10421F128E0E216F10401F154F42D
S1131490E2E0EE16F10421F5812C912CA12CB0E4AC
S11314A0BB2E3EC0FAE0EF16F10439F020E1E2165B
S11314B0F104B1F430C0103319F1FAE0EF2EF12C3D
S11314C0ACEC8A2E982CA82CACE0BA2E29C078E07B
S11314D0E72EF12C812C912CA12CE0E1BE2E20C012
S11314E060E070E080E090E897010F2C000C440B62
S11314F0550B0E94A90849015A0112C0103359F42E
S113150088818F7D883509F0BACF198122960260CF
S113151080E1E82EF12C812C912CA12C68E0B62ED0
S113152040E060E070E0CB0127010F2C000C66085E
S11315307708FE0150ED352E310E29E0231570F4A5
S11315402FEB210F2A3118F439EC332E06C02FE982
S1131550210F2A3118F529EA322E310E232D30E0DD
S11315602E153F05DCF447FD16C086169706A8061F
S1131570B90670F0A30192010E949908630D711DD0
S1131580811D911D61307105810520E8920710F0DD
S11315904FEF01C041E021961081CBCF202F217065
S11315A0C114D10471F0442329F02197F601D183A9
S11315B0C08307C001FF19C02297F601D183C083FD
S11315C014C047FF12C0222329F060E070E080E0DD
S11315D090E804C06FEF7FEF8FEF9FE722E230E0E7
S11315E03093E0022093DF0209C0222381F090951A
S11315F08095709561957F4F8F4F9F4F462F372F62
S1131600282F12C040E030E020E090E00DC097FFAA
S1131610F5CF82E290E09093E0028093DF026FEFD7
S11316207FEF8FEF9FE7EACF642F732F822FCDB721
S1131630DEB7E1E10C94240E91110C94900D8032EC
S113164019F089508550C8F708959111089581566D
S11316508A5108F48052855808950F931F93CF93AD
S1131660DF93FB01238121FD03C08FEF9FEF2CC08B
S113167022FF16C0468157812481358142175307C2
S113168044F4A081B1819D012F5F3F4F31832083BA
S11316908C93268137812F5F3F4F3783268314C075
S11316A08B01EC01FB010084F185E02D0995892B68
S11316B0E1F6D80116968D919C911797019617968D
S11316C09C938E931697CE01DF91CF911F910F912A
S11316D00895A0E0B0E0EFE6FBE00C94170EAE0135
S11316E04B5F5F4FFA0161917191AF018091DB0211
S11316F09091DC020E94AF0BE2E00C94330E0F9346
S11317001F93CF93DF93E091DB02F091DC022381FE
S113171021FF1BC08C01D0E0C0E0F80181918F0152
S11317206091DB027091DC02DB011896ED91FC9173
S11317301997882331F00995892B79F3DFEFCFEFDF
S1131740ECCF8AE00995892B19F08FEF9FEF02C047
S11317508D2F9C2FDF91CF911F910F910895ABE0B6
S1131760B0E0E5EBFBE00C94070E6C017B018A0111
S1131770FC0117821682838181FFCCC1CE010196C0
S11317803C01F6019381F70193FD859193FF8191CB
S11317907F01882309F4BAC1853239F493FD859118
S11317A093FF81917F01853229F4B60190E00E9474
S11317B02D0BE7CF912C212C312CFFE1F315D8F020
S11317C08B3279F038F4803279F08332A1F4232D0E
S11317D020611DC08D3261F0803369F4232D2160B6
S11317E016C0832D8260382EE32DE4603E2E2AC07D
S11317F0F32DF8601DC037FC2DC020ED280F2A30D2
S113180040F08E32B9F436FC81C1232D2064322E8F
S113181019C036FE06C08AE0989E200D1124922E2F
S113182011C0EAE02E9E200D1124222EF32DF06229
S11318303F2E08C08C3621F4832D8068382E02C0D8
S1131840883641F4F70193FD859193FF81917F01DF
S11318508111B3CF982F9F7D9554933028F40C5F5A
S11318601F4F9FE399830DC0833631F0833771F0A6
S1131870833509F059C021C0F801808189830E5F46
S11318801F4F88248394912C530113C02801F2E044
S11318904F0E511CF801A080B18036FE03C0692DA3
S11318A070E002C06FEF7FEFC5010E949E0D4C01F6
S11318B08201F32DFF773F2E16C0280122E0420E4D
S11318C0511CF801A080B18036FE03C0692D70E080
S11318D002C06FEF7FEFC5010E94930D4C01F32D01
S11318E0F0683F2E820133FC1BC0822D90E08816E5
S11318F09906B0F4B60180E290E00E942D0B2A9480
S1131900F4CFF50137FC859137FE81915F01B60173
S113191090E00E942D0B21102A9421E0821A910854
S11319208114910471F7E8C0843611F0893641F5C9
S1131930F80137FE07C060817181828193810C5F59
S11319401F4F08C060817181072E000C880B990B12
S11319500E5F1F4FF32DFF763F2E97FF09C0909522
S11319608095709561957F4F8F4F9F4FF0683F2E04
S11319702AE030E0A3010E94A90D882E861845C0F4
S1131980853731F4232D2F7EB22E2AE030E025C096
S1131990932D997FB92E8F36C1F018F4883579F0DC
S11319A0B5C0803719F0883721F0B0C0E92FE06165
S11319B0BE2EB4FE0DC0FB2DF460BF2E09C034FE54
S11319C00AC0292F2660B22E06C028E030E005C0E8
S11319D020E130E002C020E132E0F801B7FE07C0A8
S11319E060817181828193810C5F1F4F06C0608189
S11319F0718180E090E00E5F1F4FA3010E94A90D4A
S1131A00882E8618FB2DFF773F2E36FE0DC0232D22
S1131A102E7FA22E891458F434FE0BC032FC09C068
S1131A20832D8E7EA82E05C0B82CA32C03C0B82C01
S1131A3001C0B92CA4FE0FC0FE01E80DF11D808188
S1131A40803321F49A2D997EA92E09C0A2FE06C0E6
S1131A50B394B39404C08A2D867809F0B394A3FC9C
S1131A6011C0A0FE06C0B21488F4280C922C9B1856
S1131A700EC0B21460F4B60180E290E00E942D0B17
S1131A80B394F7CFB21418F42B1802C0982C212C5D
S1131A90A4FE10C0B60180E390E00E942D0BA2FECC
S1131AA017C0A1FC03C088E790E002C088E590E07D
S1131AB0B6010CC08A2D867859F0A1FE02C08BE2D3
S1131AC001C080E2A7FC8DE2B60190E00E942D0BDC
S1131AD0891438F4B60180E390E00E942D0B9A94A7
S1131AE0F7CF8A94F301E80DF11D8081B60190E0EF
S1131AF00E942D0B8110F5CF222009F442CEB601AD
S1131B0080E290E00E942D0B2A94F6CFF6018681A4
S1131B10978102C08FEF9FEF2B96E2E10C94230E86
S1131B20992788270895FC010590615070400110A1
S1131B30D8F7809590958E0F9F1F0895FC016150F2
S1131B40704001900110D8F7809590958E0F9F1FDB
S1131B500895FA01AA27283051F1203181F1E8943F
S1131B606F936E7F6E5F7F4F8F4F9F4FAF4FB1E08C
S1131B703ED0B4E03CD0670F781F891F9A1FA11D87
S1131B80680F791F8A1F911DA11D6A0F711D811D88
S1131B90911DA11D20D009F468943F912AE0269F4D
S1131BA011243019305D3193DEF6CF010895462FAC
S1131BB04770405D4193B3E00FD0C9F7F6CF462F8D
S1131BC04F70405D4A3318F0495D31FD40524193F6
S1131BD002D0A9F7EACFB4E0A695979587957795B3
S1131BE06795BA95C9F700976105710508959B013A
S1131BF0AC010A2E06945795479537952795BA95C3
S1131C00C9F7620F731F841F951FA01D08952F929B
S1131C103F924F925F926F927F928F929F92AF9278
S1131C20BF92CF92DF92EF92FF920F931F93CF93C5
S1131C30DF93CDB7DEB7CA1BDB0B0FB6F894DEBF5C
S1131C400FBECDBF09942A88398848885F846E8482
S1131C507D848C849B84AA84B984C884DF80EE80CC
S1131C60FD800C811B81AA81B981CE0FD11D0FB6D5
S1131C70F894DEBF0FBECDBFED010895F894FFCFF9
S1131C800000E1022000FFFFFFFF0000000200004F
S1131C9000008C08000000006C017001436F6E7638
S1131CA04669666F004572726F72204932435F5312
S1131CB054415254004572726F72204932435F534B
S1131CC04C415F41434B004572726F72204932436D
S1131CD05F444154415F41434B0053657420737723
S1131CE06974636820746F2025730A004F464600A8
S1131CF04F4E0053657420506F77657220746F20C7
S1131D002575206469676974730A00257320257337
S1131D100A004F4B3A25303475004552523A496E09
S1131D2076616C6964207374617465004F4B3A2565
S1131D3075004F4B3A2564004F4B3A2573004552CA
S1131D40523A556E6B6E6F776E20636F6D6D616E78
S1131D50640052656D6F74652074696D656F757488
S1131D6021005077725377697463685F696E203D10
S1131D702025640A005374617465206368616E678A
S1131D80652022257322203D3E20222573220A004D
S1131D904E6F726D616C0052656D6F7465005375A2
S1131DA07370656E64004572726F720010021702E0
S1131DB01E02260276312E31340048656E64692D88
S1131DC0436F6E74726F6C000502010B06010B0702
S1131DD0010B02010B03010B04010B0501050101B9
S9030000FC
